S021000064656D6F70726F675F6F6C696D65785F73746D3332703130332E737265639D
S3150800600000500020696D0008B96D0008B96D0008D8
S31508006010B96D0008B96D0008B96D000800000000E8
S31508006020000000000000000000000000B96D000834
S31508006030B96D000800000000B96D0008016E00087F
S31508006040B96D0008B96D0008B96D0008B96D00088A
S31508006050B96D0008B96D0008B96D0008B96D00087A
S31508006060B96D0008B96D0008B96D0008B96D00086A
S31508006070B96D0008B96D0008B96D0008B96D00085A
S31508006080B96D0008B96D0008B96D0008B96D00084A
S31508006090B96D0008B96D0008B96D0008B96D00083A
S315080060A0B96D0008B96D0008B96D0008B96D00082A
S315080060B0B96D0008B96D0008B96D0008B96D00081A
S315080060C0B96D0008B96D0008B96D0008B96D00080A
S315080060D0B96D0008B96D0008B96D0008B96D0008FA
S315080060E0B96D0008B96D0008B96D00080000000018
S315080060F00000000000000000000000000000000092
S3150800610000000000000000005FF808F111EEAA5533
S3150800611010B5054C237833B9044B13B10448AFF3D3
S3150800612000800123237010BD140000200000000029
S31508006130586E000808B5034B1BB103490348AFF373
S31508006140008008BD0000000018000020586E0008F6
S31508006150F0B5002401E00134E4B2112C20D8114D29
S3150800616015F8147005EB440595F801E007EB0E05E4
S3150800617005FB000548F6A04C9CFBF5F605FB16C684
S31508006180002EE8D19CFBF5F5ADB20D80013DADB210
S31508006190B5F5806FDFD2177083F800E00120F0BDF7
S315080061A00020F0BD706E000830B587B001214FF4AD
S315080061B0003000F0B3FC0121052000F0A1FC1823F3
S315080061C08DF817300425ADF8145003238DF81630D2
S315080061D0144C05A9204600F0A8FB8DF81750082393
S315080061E0ADF8143005A9204600F09FFB4FF4614333
S315080061F001930023ADF80830ADF80A30ADF80C303D
S31508006200ADF810300C23ADF80E30A4F544440DEB70
S315080062100501204600F09EFC0121204600F0FEFC08
S3150800622007B030BD0008014030B58BB001210846E3
S3150800623000F066FC0121082000F062FC4FF4807330
S31508006240ADF8243048238DF82730344C09A9204668
S3150800625000F06BFB4FF40073ADF8243018238DF86B
S31508006260273003238DF8263009A9204600F05DFB68
S3150800627001214FF4EA1000F0ABFB01214FF000704A
S3150800628000F04CFC264D284600F0BEF906A800F0A2
S31508006290DDFA01AB0DF105020DF106014FF4FA70B6
S315080062A0FFF756FF00248DF81E408DF81F408DF825
S315080062B020408DF821408DF822408DF823408DF836
S315080062C01A408DF81B409DF80530013B8DF81C30AF
S315080062D09DF80430013B8DF81D30BDF80630ADF849
S315080062E0183006A9284600F0ABF98DF812408DF84B
S315080062F0134001238DF81430ADF80840ADF80A4074
S31508006300ADF80C40ADF80E40ADF810408DF81530DC
S3150800631002A800F01DFA0BB030BD00BF000C01400A
S315080063200064004010B504462021064800F088FCA9
S31508006330012801D0002010BD024800F07DFC207025
S31508006340012010BD0044004008B5FFF72DFFFFF7F8
S315080063506BFF08BD0449CA6802F4E062034B1343A5
S31508006360CB60BFF34F8FFEE700ED00E00400FA05AF
S3150800637008B5224B1B78B3B92148FFF7D3FF01288C
S3150800638000D008BD1E4B1B78013BDBB23F2BF8D86B
S3150800639000F030FD1B4B18600122184B1A700022C2
S315080063A0194B1A7008BD184B1B780133144818444A
S315080063B0FFF7B8FF01280AD000F01CFD114B1B6837
S315080063C064339842DDD900220C4B1A70D9E70E4A7D
S315080063D013780133DBB21370094A12789342D0D18D
S315080063E00022064B1A70064B5B78FF2BC9D1044B6B
S315080063F09B78002BC5D1FFF7ADFF00BF71000020C9
S3150800640030000020740000207200002000B587B01C
S315080064100021124800F07CFA10B907B05DF804FBB9
S3150800642001AA00210D4800F021FA9DF80C3033B975
S3150800643040F26763019A9A420ED0002300E00023D7
S31508006440002BEAD09DF80F30FF2BE6D19DF81030CF
S31508006450002BE2D1FFF77EFF0123F1E7006400403D
S3150800646008B5FFF785FFFFF7D1FF08BD30B583B044
S315080064700121102000F044FB4FF48055ADF804507C
S3150800648003238DF8063010238DF80730054C01A933
S31508006490204600F04AFA2946204600F095FA03B04D
S315080064A030BD00BF0010014010B500F0A3FC0F4B33
S315080064B01B68C31AB3F5FA7F0DD304460C4B1B7839
S315080064C053B901220A4B1A704FF48051094800F05B
S315080064D07DFA064B1C6010BD0022054B1A704FF45E
S315080064E08051044800F070FAF3E700BF7C000020F2
S315080064F0780000200010014082B000230193009329
S315080065002C4A136843F4803313602A4B1B6803F440
S3150800651000330093019B01330193009B1BB9019B38
S31508006520B3F5A06FF1D1234B1B6813F4003F06D0D7
S3150800653001230093009B012B04D002B0704700236F
S315080065400093F7E71C4B1A6842F010021A601A68A3
S3150800655022F003021A601A6842F002021A60A3F5D2
S3150800656080535A685A605A685A605A6842F4806278
S315080065705A605A6822F47C125A605A6842F4E81241
S315080065805A601A6842F080721A600A4B1B6813F048
S31508006590007FFAD0074B5A6822F003025A605A68FD
S315080065A042F002025A60034B5B6803F00C03082BA7
S315080065B0F9D1C2E7001002400020024008B5FFF7F3
S315080065C09BFF08BD08B50E4B1A6842F001021A6017
S315080065D059680C4A0A405A601A6822F0847222F4F2
S315080065E080321A601A6822F480221A605A6822F4E5
S315080065F0FE025A604FF41F029A60FFF7DFFF08BDDC
S31508006600001002400000FFF808B50C4B98420AD06B
S3150800661001214FF0806000F08FFA00214FF0806072
S3150800662000F08AFA08BD01214FF0007000F084FAE4
S3150800663000214FF0007000F07FFA08BD00640040AA
S31508006640036823F002030360036843F00103036051
S31508006650002300E00133426812F0010F03D14FF620
S31508006660FF729342F6D1436813F0010F6DD08B7910
S31508006670012B3BD0036823F080030360CB79012B01
S3150800668039D0036823F0400303600B7A012B37D017
S31508006690036823F0200303604B7A012B35D0036887
S315080066A023F0100303608B7A012B33D0036823F0A1
S315080066B008030360CB7A012B31D0036823F0040367
S315080066C003608A78CB781B0643EA82730A7943EA21
S315080066D002434A7943EA02530A88013A1343C361DB
S315080066E0036823F00103036000231EE0036843F0F8
S315080066F080030360C2E7036843F040030360C4E70E
S31508006700036843F020030360C6E7036843F01003F9
S315080067100360C8E7036843F008030360CAE7036831
S3150800672043F004030360CCE70133426812F0010F1B
S3150800673003D04FF6FF729342F6D1436813F0010F68
S3150800674001D10120704700207047002070470000E3
S3150800675070B4837A012202FA03F33B4AD2F8001294
S3150800676041F00101C2F80012D2F81C42D9430C408C
S31508006770C2F81C42027BB2B9334AD2F80C420C402A
S31508006780C2F80C42847AC688458845EA06454834E4
S3150800679042F83450857A8688048844EA064448359F
S315080067A002EBC5025460027B012A1FD0C27A002A76
S315080067B034D1254CD4F804220A40C4F804220289AC
S315080067C02AB9214AD2F814422140C2F81412028981
S315080067D0012A2AD0427B012A2ED01B4AD2F800323F
S315080067E023F00103C2F8003270BC7047164AD2F88B
S315080067F00C421C43C2F80C42847A0688458845EA4E
S315080068000645483442F83450857A8688C48844EA6E
S315080068100644483502EBC5025460C7E70A4CD4F86B
S3150800682004221A43C4F80422C9E70749D1F81422F6
S315080068301A43C1F81422CDE7034AD2F81C120B43B7
S31508006840C2F81C32C9E700BF006400400023837108
S31508006850C371037243728372C3728370C370032356
S3150800686003710223437101230380704710B401F1B9
S315080068701B031B01C35803F004031372002B3BD1FF
S3150800688001F11B031B01C3585B0D136001F11B03C8
S315080068901B01C418C35803F002035372636803F05C
S315080068A00F03937263681B0AD37400EB0113D3F8C2
S315080068B0B841D472D3F8B841240A1473D3F8B8414E
S315080068C0240C5473D3F8B841240E9473D3F8BC41FE
S315080068D0D473D3F8BC41240A1474D3F8BC41240CED
S315080068E05474D3F8BC311B0E937461B1036943F039
S315080068F02003036110BC704701F11B031B01C35839
S31508006900DB085360C2E7C36843F02003C360F1E7BE
S3150800691019B1012905D000207047C06800F00300AE
S315080069207047006900F003007047F0B4CB7803F0B5
S315080069300F02154613F0100F01D08D7815430B780A
S31508006940E3B10668002301E042610133072B14D83E
S3150800695001229A400C8832EA0404F6D19C000F27DB
S31508006960A74026EA070605FA04F42643CC78282C1D
S31508006970EAD0482CE9D10261E7E706600B88FF2BCD
S3150800698020D94668002302E0426115E00133072B4F
S3150800699017D803F108040122A2400C8832EA04043D
S315080069A0F4D19C000F27A74026EA070605FA04F447
S315080069B02643CC78282CE7D0CC78482CE6D102613F
S315080069C0E4E74660F0BC7047016170474161704773
S315080069D030B400281DDB1A4B5B68C0F3034582B24E
S315080069E000F44014B4F5401F16D010F4801F1BD0D5
S315080069F00324AC4023EA040343F0706319B1410D44
S31508006A0009018A401343002817DB0D4A536030BC3E
S31508006A1070470B4BDB69E0E723F07063084D6C6841
S31508006A2024F070646C60E9E7440D240102FA04F46A
S31508006A3023EA040343F07063E0E7014AD361E6E71B
S31508006A400000014010B4294B5B6803F00C03042BCB
S31508006A502BD0082B2CD013B1254B036001E0244B17
S31508006A60036022494B68C3F30313224CE35CDAB292
S31508006A700368D34043604A68C2F30222A25CD2B2DA
S31508006A8023FA02F282604A68C2F3C222A25CD2B238
S31508006A90D340C3604A68C2F3813217498A5CD2B2CE
S31508006AA0B3FBF2F3036110BC7047114B0360D8E7E0
S31508006AB00E4A53685268C3F38343023312F4803F85
S31508006AC009D00A4A526812F4003F09D00B4A02FB61
S31508006AD003F30360C5E7094A02FB03F30360C0E753
S31508006AE0034A02FB03F30360BBE700BF0010024042
S31508006AF000127A00040000200000002000093D0072
S31508006B0029B9054A936923EA000090617047024A49
S31508006B1093691843906170470010024029B9054AE5
S31508006B20D36923EA0000D0617047024AD369184343
S31508006B30D06170470010024029B9054A136923EA53
S31508006B40000010617047024A1369184310617047C4
S31508006B500010024030B587B004460D46038A9BB242
S31508006B60CA8823F440531343038283899BB28988D6
S31508006B7028896A8901430A4323F4B05323F00C0396
S31508006B801343A381A38A9BB2AA8923F440731343B0
S31508006B90A38201A8FFF756FF1E4B9C4224D0039BF5
S31508006BA0A28912F4004F21D103EB830303EB83037D
S31508006BB029688900B3FBF1F1174BA3FB0123580998
S31508006BC00501642300FB1313A28912F4004F16D1A2
S31508006BD01B013233104AA2FB0323C3F343132B438F
S31508006BE09BB2238107B030BD049BD9E703EB83032F
S31508006BF003EB830329684900B3FBF1F1DCE7D9000D
S31508006C003231054AA2FB0131C1F3421245EA0203B9
S31508006C10E6E700BF003801401F85EB5131B983898B
S31508006C209BB223F400539BB28381704783899BB23E
S31508006C3043F40053838170478088C0F30800704787
S31508006C400388194201D100207047012070470000CF
S31508006C5000B583B000230193009303F1804303F545
S31508006C6004331A6842F001021A605968364A0A4023
S31508006C705A601A6822F0847222F480321A601A68FE
S31508006C8022F480221A605A6822F4FE025A604FF4EF
S31508006C901F029A601A6842F480321A602B4B1B68EE
S31508006CA003F400330093019B01330193009B23B93E
S31508006CB0019A40F2DC539A42F0D1244B1B6813F434
S31508006CC0003F00D1FEE7224B1A6842F010021A6014
S31508006CD01A6822F003021A601A6842F002021A6061
S31508006CE0A3F580535A685A605A6842F400525A60AB
S31508006CF05A6842F480625A605A6822F47C125A60D2
S31508006D005A6842F4E8125A601A6842F080721A60A9
S31508006D100E4B1B6813F0007FFAD00C4B5A6822F012
S31508006D2003025A605A6842F002025A60074B5B68CF
S31508006D3003F00C03082BF9D1FFF798FB00F044F891
S31508006D4003B05DF804FB00BF0000FFF80010024026
S31508006D500020024008B5FFF77BFFFFF7F5FAFFF7BB
S31508006D60A3FBFFF77DFBFAE7DFF834D0002103E049
S31508006D700C4B5B58435004310B480C4B42189A4253
S31508006D80F6D30B4A02E0002342F8043B094B9A4229
S31508006D90F9D3FFF717FC00F03BF8FFF7DBFF704766
S31508006DA0005000209C6E00080000002014000020FF
S31508006DB01400002084000020FEE70000014B186044
S31508006DC0704700BF8000002008B5074B074A5A6085
S31508006DD0F021074A82F823100020986007221A60DB
S31508006DE0FFF7ECFF08BD00BF10E000E03F19010007
S31508006DF000ED00E0014B1868704700BF80000020D6
S31508006E00024A136801331360704700BF80000020F0
S31508006E1070B500250C4E0D4CA41BA410A54209D133
S31508006E2000F01AF800250A4E0A4CA41BA410A54225
S31508006E3005D170BD56F8253098470135EEE756F866
S31508006E40253098470135F2E7946E0008946E0008DD
S31508006E50946E0008986E0008F8B500BFF8BC08BC28
S31508006E609E467047F8B500BFF8BC08BC9E467047FA
S31508006E7005020602060307030803090309040A04B0
S31508006E800B040C040C050D050E050F050F06100660
S30908006E9010071008C1
S30908006E94356100084E
S30908006E98116100086E
S31508006E9C02040608000000000102030401020304B0
S30908006EAC06070809B6
S70508006D691C
